:020000040000FA
:100000000D290408A2008316051283120930A300EB
:1000100003101120A20CA30B0928031411200314B0
:100020000829031816280000051618280512182894
:100030000030A1006230B728B31329080319B317A1
:100040000530A8002730A300103032200330A30071
:10005000E8303220A30164303220A3010A3032207C
:1000600024083928A2002508A1002408A000E720C0
:100070002008A000A8030319B31329080319432873
:100080002802031808002008031DB313B31B08003F
:10009000303E0329A3003608840034097E208413EF
:1000A000A30803190829F030A50022088038A4000D
:1000B000F030A5030319A5000319A30303190829A8
:1000C0002008A6002108A7001630B6202608A000A8
:1000D0002708A1009A20030120183408A21F340821
:1000E000A20803190301A40F772880065528782851
:1000F000000058288120FF3A80057E28841780055B
:100100000829A8000530A8190730840000308A00AB
:1001100028080739820701340234043408341034C3
:1001200020344034803483178001840AFF3E031D4D
:1001300094280829210820040319A00A8030201AD5
:10014000A1062019A106A018A106210DA00DA10D40
:100150000829A301A200FF30A207031CA307031C68
:1001600008290330A100E330B720AB28A101F43EF9
:10017000A000A109FE30031CC028A0070318BD2859
:10018000A0076400A10FBD2800002018C728201870
:10019000C9280800013EA7000A30A200A301E720F9
:1001A000A70BCF2824080800A2000130D728A800F8
:1001B00023082102031DDE28220820020430031830
:1001C0000130031902302805031DFF300829A5015D
:1001D000A4011030A600210DA40DA50D2208A40233
:1001E0002308031C230FA5020318FD282208A407D7
:1001F00023080318230FA5070310A00DA10DA60BBC
:10020000EB2820080829840031088A003008820081
:1002100083130313831264000800831690017E3059
:100220008F0083128B010F3099008316991383126C
:1002300083169F0183129F01831691010B30850065
:10024000870120308400603083128A019420A0301E
:10025000840050308A0194202030840050308A017C
:1002600093200516831605120D3083128A01022091
:100270000A308A0102200D308A0102200A308A01E8
:10028000022032308A01A92045308A0102204C30F8
:100290008A01022045308A01022043308A0102206F
:1002A00054308A01022052308A0102204F308A01E4
:1002B00002204E308A01022049308A010220433058
:1002C0008A01022020308A01022044308A01022063
:1002D00049308A01022043308A01022045308A01D8
:1002E00002200D308A0102200A308A0102200D30DE
:1002F0008A0102200A308A01022056308A01022037
:1003000031308A0102202E308A01022030308A01E9
:1003100002200D308A0102200A308A0102200D30AD
:100320008A0102200A308A0102200D308A0102204F
:100330000A308A0102204D308A01022041308A01B0
:10034000022044308A01022045308A0102202030F8
:100350008A01022042308A01022059308A0102209B
:1003600020308A01022052308A01022055308A0151
:10037000022049308A01022020308A0102204330C5
:100380008A01022041308A01022042308A01022083
:1003900052308A01022041308A0102204C308A0109
:1003A000022020308A01022032308A0102203030BF
:1003B0008A01022031308A01022030308A01022075
:1003C0000D308A0102200A308A0102200D308A0194
:1003D00002200A308A0102200D308A0102200A30F0
:1003E0008A01022007088A017A2005118316051167
:1003F00005308312B6002030B4007D30A2000530F5
:100400008A014A207D30A20005308A014A208701F6
:1004100064308A01A9200130870064308A01A92054
:100420000330870064308A01A920073087006430D8
:100430008A01A9200F30870064308A01A9201F306B
:10044000870064308A01A9203F30870064308A0128
:10045000A920051583160511643083128A01A9208D
:10046000051183160511643083128A01A9201F30FB
:10047000870064308A01A9200F30870064308A0128
:10048000A9200730870064308A01A9200330870043
:1004900064308A01A9200130870064308A01A920D4
:1004A000870164308A01A9200530B6002030B400ED
:1004B0007D30A20005308A014A207D30A20005303F
:1004C0008A014A2032308A01A920C8014608A000CA
:1004D0004708A1008A019A202008C6002108C70009
:1004E00064008A11851D762A8A11242BA9014608E9
:1004F000A4004708A5000130B000B1018A011C200A
:100500000D308A0102200A308A0102208A01652A00
:1005100052308A01022045308A01022053308A017C
:10052000022055308A0102204C308A0102205430CA
:100530008A01022041308A01022044308A010220CF
:100540004F308A01022020308A01022046308A0181
:10055000022049308A0102204E308A0102204130B7
:100560008A0102204C308A01022020308A010220B8
:100570003D308A01022020308A0102202E308A017B
:1005800002202E308A0102202E308A0102202030E3
:100590008A010220A9014808A400A5010130B00089
:1005A000B1018A011C200D308A0102200A308A0123
:1005B00002200D308A0102200A308A0102206400E4
:1005C0004808013C8A11031DE72A870105156400CC
:1005D0004808023C8A11031DF02A093087000511E2
:1005E00064004808033C8A11031DF92A093087007A
:1005F000051564004808043C8A11031D022B2D30A8
:100600008700051164004808053C8A11031D0B2B67
:100610002D308700051564004808063C8A11031D2B
:10062000142B3F30870005110530B6002030B40090
:100630007D30A20005308A014A207D30A2000530BD
:100640008A014A208A11FD2BBE01BF01BE01BF01F4
:100650003E08A0003F08A100A3010A308A01D4206F
:100660008A11031D4A2B64008A11851D392B8A01CA
:10067000242B0530B6002030B4007D30A2000230BB
:100680008A014A208A114C23BE0A0319BF0A8A1123
:10069000031D282B8A11702B8701051532308A0122
:1006A000A92009308700051132308A01A9200930BC
:1006B0008700051532308A01A9202D3087000511E9
:1006C00032308A01A9202D308700051532308A0189
:1006D000A9203F30870005110A308A01A9200800AF
:1006E0004608A0004708A10000308A01CA20C800BF
:1006F000A9014608A4004708A5000130B000B101D7
:100700008A011C200D308A0102200A308A01022051
:1007100052308A01022045308A01022053308A017A
:10072000022055308A0102204C308A0102205430C8
:100730008A01022041308A01022044308A010220CD
:100740004F308A01022020308A01022043308A0182
:10075000022041308A0102204C308A0102204330BD
:100760008A01022055308A0102204C308A01022081
:1007700041308A01022044308A0102204F308A0130
:10078000022020308A0102203D308A0102202030E0
:100790008A0102202E308A0102202E308A01022096
:1007A0002E308A01022020308A010220A901480847
:1007B000A400A5010130B000B1018A011C200D3058
:1007C0008A0102200A308A0102200D308A010220AB
:1007D0000A308A0102206400083048028A11031C92
:1007E000F32B0330C8026400013048028A11031859
:1007F000FB2B0230C8008A01882A0330A300E830AE
:0E0800008A01AA208A01652A63008A01042C5D
:02400E00FC3F75
:00000001FF
